******************************************************************************
                  TI ARM Linker PC v16.9.6                     
******************************************************************************
>> Linked Wed May 09 14:30:30 2018

OUTPUT FILE NAME:   <BSL_TEST.out>
ENTRY POINT SYMBOL: "_c_int00"  address: 00000a7d


MEMORY CONFIGURATION

         name            origin    length      used     unused   attr    fill
----------------------  --------  ---------  --------  --------  ----  --------
  MAIN                  00000000   00040000  00000cb0  0003f350  R  X
  INFO                  00200000   00004000  00000000  00004000  R  X
  SRAM_CODE             01000000   00010000  00000314  0000fcec  RW X
  SRAM_DATA             20000000   00010000  00000314  0000fcec  RW  


SEGMENT ALLOCATION MAP

run origin  load origin   length   init length attrs members
----------  ----------- ---------- ----------- ----- -------
00000000    00000000    00000cb0   00000cb0    r-x
  00000000    00000000    000000e4   000000e4    r-- .intvecs
  000000e4    000000e4    00000b74   00000b74    r-x .text
  00000c58    00000c58    00000008   00000008    r-- .const
  00000c60    00000c60    00000050   00000050    r-- .cinit
20000000    20000000    00000114   00000000    rw-
  20000000    20000000    000000e8   00000000    rw- .vtable
  200000e8    200000e8    00000024   00000000    rw- .data
  2000010c    2000010c    00000008   00000000    rw- .bss
2000fe00    2000fe00    00000200   00000000    rw-
  2000fe00    2000fe00    00000200   00000000    rw- .stack


SECTION ALLOCATION MAP

 output                                  attributes/
section   page    origin      length       input sections
--------  ----  ----------  ----------   ----------------
.intvecs   0    00000000    000000e4     
                  00000000    000000e4     startup_msp432p401r_ccs.obj (.intvecs:retain)

.binit     0    00000000    00000000     

.text      0    000000e4    00000b74     
                  000000e4    00000374     main.obj (.text)
                  00000458    00000334     system_msp432p401r.obj (.text)
                  0000078c    0000009c     msp432p4xx_driverlib.lib : cs_MSP432P4XX.obj (.text:CS_startLFXTWithTimeout)
                  00000828    0000009c     rtsv7M4_T_le_v4SPD16_eabi.lib : memcpy_t2.obj (.text)
                  000008c4    0000007a                                   : memset_t2.obj (.text)
                  0000093e    00000002                                   : mpu_init.obj (.text)
                  00000940    00000070                                   : autoinit.obj (.text)
                  000009b0    00000068                                   : copy_decompress_lzss.obj (.text:decompress:lzss)
                  00000a18    00000064     msp432p4xx_driverlib.lib : interrupt_MSP432P4XX.obj (.text:Interrupt_enableInterrupt)
                  00000a7c    00000054     rtsv7M4_T_le_v4SPD16_eabi.lib : boot.obj (.text)
                  00000ad0    00000054                                   : exit.obj (.text)
                  00000b24    0000004c                                   : cpy_tbl.obj (.text)
                  00000b70    00000034     msp432p4xx_driverlib.lib : interrupt_MSP432P4XX.obj (.text:Interrupt_registerInterrupt)
                  00000ba4    00000018     rtsv7M4_T_le_v4SPD16_eabi.lib : args_main.obj (.text)
                  00000bbc    00000014     msp432p4xx_driverlib.lib : cs_MSP432P4XX.obj (.text:CS_setExternalClockSourceFrequency)
                  00000bd0    00000014     rtsv7M4_T_le_v4SPD16_eabi.lib : _lock.obj (.text)
                  00000be4    00000010     msp432p4xx_driverlib.lib : sysctl_a_MSP432P4XX.obj (.text:SysCtl_A_disableNMISource)
                  00000bf4    00000010                              : sysctl_a_MSP432P4XX.obj (.text:SysCtl_A_enableNMISource)
                  00000c04    00000010                              : sysctl_a_MSP432P4XX.obj (.text:SysCtl_A_getNMISourceStatus)
                  00000c14    00000010                              : timer32_MSP432P4XX.obj (.text:Timer32_registerInterrupt)
                  00000c24    0000000e     rtsv7M4_T_le_v4SPD16_eabi.lib : copy_decompress_none.obj (.text:decompress:none)
                  00000c32    0000000e     startup_msp432p401r_ccs.obj (.text)
                  00000c40    0000000c     rtsv7M4_T_le_v4SPD16_eabi.lib : copy_zero_init.obj (.text:decompress:ZI)
                  00000c4c    00000006     msp432p4xx_driverlib.lib : cs_MSP432P4XX.obj (.text:CS_startLFXT)
                  00000c52    00000004     rtsv7M4_T_le_v4SPD16_eabi.lib : pre_init.obj (.text)
                  00000c56    00000002                                   : startup.obj (.text)

.const     0    00000c58    00000008     
                  00000c58    00000008     msp432p4xx_driverlib.lib : interrupt_MSP432P4XX.obj (.const:g_pulEnRegs)

.cinit     0    00000c60    00000050     
                  00000c60    00000015     (.cinit..data.load) [load image, compression = lzss]
                  00000c75    00000003     --HOLE-- [fill = 0]
                  00000c78    0000000c     (__TI_handler_table)
                  00000c84    00000004     --HOLE-- [fill = 0]
                  00000c88    00000008     (.cinit..bss.load) [load image, compression = zero_init]
                  00000c90    00000008     (.cinit..vtable.load) [load image, compression = zero_init]
                  00000c98    00000018     (__TI_cinit_table)

.init_array 
*          0    00000000    00000000     UNINITIALIZED

.vtable    0    20000000    000000e8     UNINITIALIZED
                  20000000    000000e8     msp432p4xx_driverlib.lib : interrupt_MSP432P4XX.obj (.vtable)

.data      0    200000e8    00000024     UNINITIALIZED
                  200000e8    0000000c     rtsv7M4_T_le_v4SPD16_eabi.lib : exit.obj (.data:$O1$$)
                  200000f4    00000008                                   : _lock.obj (.data:$O1$$)
                  200000fc    00000005     main.obj (.data)
                  20000101    00000003     --HOLE--
                  20000104    00000004     rtsv7M4_T_le_v4SPD16_eabi.lib : stkdepth_vars.obj (.data)
                  20000108    00000004     system_msp432p401r.obj (.data)

.bss       0    2000010c    00000008     UNINITIALIZED
                  2000010c    00000008     msp432p4xx_driverlib.lib : cs_MSP432P4XX.obj (.bss)

.stack     0    2000fe00    00000200     UNINITIALIZED
                  2000fe00    00000200     --HOLE--

MODULE SUMMARY

       Module                        code   ro data   rw data
       ------                        ----   -------   -------
    .\
       main.obj                      884    0         10     
       system_msp432p401r.obj        820    0         8      
       startup_msp432p401r_ccs.obj   14     228       0      
    +--+-----------------------------+------+---------+---------+
       Total:                        1718   228       18     
                                                             
    C:/ti/simplelink_msp432p4_sdk_1_60_00_12/source/ti/devices/msp432p4xx/driverlib/ccs/msp432p4xx_driverlib.lib
       interrupt_MSP432P4XX.obj      152    8         464    
       cs_MSP432P4XX.obj             182    0         16     
       sysctl_a_MSP432P4XX.obj       48     0         0      
       timer32_MSP432P4XX.obj        16     0         0      
    +--+-----------------------------+------+---------+---------+
       Total:                        398    8         480    
                                                             
    C:\ti\ccsv7\tools\compiler\ti-cgt-arm_16.9.6.LTS\lib\rtsv7M4_T_le_v4SPD16_eabi.lib
       memcpy_t2.obj                 156    0         0      
       memset_t2.obj                 122    0         0      
       autoinit.obj                  112    0         0      
       exit.obj                      84     0         24     
       copy_decompress_lzss.obj      104    0         0      
       boot.obj                      84     0         0      
       cpy_tbl.obj                   76     0         0      
       _lock.obj                     20     0         16     
       args_main.obj                 24     0         0      
       copy_decompress_none.obj      14     0         0      
       copy_zero_init.obj            12     0         0      
       stkdepth_vars.obj             0      0         8      
       pre_init.obj                  4      0         0      
       mpu_init.obj                  2      0         0      
       startup.obj                   2      0         0      
    +--+-----------------------------+------+---------+---------+
       Total:                        816    0         48     
                                                             
       Stack:                        0      0         1024   
       Linker Generated:             0      73        0      
    +--+-----------------------------+------+---------+---------+
       Grand Total:                  2932   309       1570   


LINKER GENERATED COPY TABLES

__TI_cinit_table @ 00000c98 records: 3, size/record: 8, table size: 24
	.data: load addr=00000c60, load size=00000015 bytes, run addr=200000e8, run size=00000024 bytes, compression=lzss
	.bss: load addr=00000c88, load size=00000008 bytes, run addr=2000010c, run size=00000008 bytes, compression=zero_init
	.vtable: load addr=00000c90, load size=00000008 bytes, run addr=20000000, run size=000000e8 bytes, compression=zero_init


LINKER GENERATED HANDLER TABLE

__TI_handler_table @ 00000c78 records: 3, size/record: 4, table size: 12
	index: 0, handler: __TI_zero_init
	index: 1, handler: __TI_decompress_lzss
	index: 2, handler: __TI_decompress_none


GLOBAL SYMBOLS: SORTED ALPHABETICALLY BY Name 

address   name                              
-------   ----                              
00000c3f  ADC14_IRQHandler                  
00000c3f  AES256_IRQHandler                 
00000c3f  BusFault_Handler                  
00000ad1  C$$EXIT                           
00000c3f  COMP_E0_IRQHandler                
00000c3f  COMP_E1_IRQHandler                
00000c3f  CS_IRQHandler                     
00000bbd  CS_setExternalClockSourceFrequency
00000c4d  CS_startLFXT                      
0000078d  CS_startLFXTWithTimeout           
00000c3f  DMA_ERR_IRQHandler                
00000c3f  DMA_INT0_IRQHandler               
00000c3f  DMA_INT1_IRQHandler               
00000c3f  DMA_INT2_IRQHandler               
00000c3f  DMA_INT3_IRQHandler               
00000c3f  DebugMon_Handler                  
00000c3f  Default_Handler                   
00000c3f  EUSCIA0_IRQHandler                
00000c3f  EUSCIA1_IRQHandler                
00000c3f  EUSCIA2_IRQHandler                
00000c3f  EUSCIA3_IRQHandler                
00000c3f  EUSCIB0_IRQHandler                
00000c3f  EUSCIB1_IRQHandler                
00000c3f  EUSCIB2_IRQHandler                
00000c3f  EUSCIB3_IRQHandler                
00000c3f  FLCTL_IRQHandler                  
00000c3f  FPU_IRQHandler                    
00000c3f  HardFault_Handler                 
00000a19  Interrupt_enableInterrupt         
00000b71  Interrupt_registerInterrupt       
00000c3f  MemManage_Handler                 
00000c3f  NMI_Handler                       
00000c3f  PCM_IRQHandler                    
0000010b  PORT1_IRQHandler                  
0000010b  PORT1_IRQHandler                  
00000c3f  PORT2_IRQHandler                  
00000c3f  PORT3_IRQHandler                  
00000c3f  PORT4_IRQHandler                  
00000c3f  PORT5_IRQHandler                  
00000c3f  PORT6_IRQHandler                  
00000c3f  PSS_IRQHandler                    
00000c3f  PendSV_Handler                    
00000c3f  RTC_C_IRQHandler                  
00000c33  Reset_Handler                     
UNDEFED   SHT$$INIT_ARRAY$$Base             
UNDEFED   SHT$$INIT_ARRAY$$Limit            
00000c3f  SVC_Handler                       
00000be5  SysCtl_A_disableNMISource         
00000bf5  SysCtl_A_enableNMISource          
00000c05  SysCtl_A_getNMISourceStatus       
00000c3f  SysTick_Handler                   
20000108  SystemCoreClock                   
00000459  SystemCoreClockUpdate             
000006d1  SystemInit                        
00000c3f  T32_INT1_IRQHandler               
00000c3f  T32_INT2_IRQHandler               
00000c3f  T32_INTC_IRQHandler               
00000c3f  TA0_0_IRQHandler                  
00000c3f  TA0_N_IRQHandler                  
00000c3f  TA1_0_IRQHandler                  
00000c3f  TA1_N_IRQHandler                  
00000c3f  TA2_0_IRQHandler                  
00000c3f  TA2_N_IRQHandler                  
00000c3f  TA3_0_IRQHandler                  
00000c3f  TA3_N_IRQHandler                  
000000e5  Timer32_0_INT                     
00000c15  Timer32_registerInterrupt         
00000c3f  UsageFault_Handler                
4000480c  WDTCTL_SYM                        
00000c3f  WDT_A_IRQHandler                  
20010000  __STACK_END                       
00000200  __STACK_SIZE                      
00000c98  __TI_CINIT_Base                   
00000cb0  __TI_CINIT_Limit                  
00000c78  __TI_Handler_Table_Base           
00000c84  __TI_Handler_Table_Limit          
00000941  __TI_auto_init                    
200000e8  __TI_cleanup_ptr                  
000009b1  __TI_decompress_lzss              
00000c25  __TI_decompress_none              
200000ec  __TI_dtors_ptr                    
200000f0  __TI_enable_exit_profile_output   
ffffffff  __TI_pprof_out_hndl               
ffffffff  __TI_prof_data_size               
ffffffff  __TI_prof_data_start              
00000000  __TI_static_base__                
00000c41  __TI_zero_init                    
000008c5  __aeabi_memclr                    
000008c5  __aeabi_memclr4                   
000008c5  __aeabi_memclr8                   
00000829  __aeabi_memcpy                    
00000829  __aeabi_memcpy4                   
00000829  __aeabi_memcpy8                   
000008c7  __aeabi_memset                    
000008c7  __aeabi_memset4                   
000008c7  __aeabi_memset8                   
ffffffff  __binit__                         
ffffffff  __c_args__                        
0000093f  __mpu_init                        
2000fe00  __stack                           
00000ba5  _args_main                        
00000a7d  _c_int00                          
200000f4  _lock                             
00000bdf  _nop                              
00000bd7  _register_lock                    
00000bd1  _register_unlock                  
00000c57  _system_post_cinit                
00000c53  _system_pre_init                  
200000f8  _unlock                           
00000ad5  abort                             
ffffffff  binit                             
00000b25  copy_in                           
00000add  exit                              
20000000  g_pfnRAMVectors                   
00000000  interruptVectors                  
0000031b  main                              
20000104  main_func_sp                      
00000829  memcpy                            
000008cd  memset                            
00000131  port_init                         
20000100  status                            
200000fc  timer                             
000002bb  timer32_init                      


GLOBAL SYMBOLS: SORTED BY Symbol Address 

address   name                              
-------   ----                              
00000000  __TI_static_base__                
00000000  interruptVectors                  
000000e5  Timer32_0_INT                     
0000010b  PORT1_IRQHandler                  
0000010b  PORT1_IRQHandler                  
00000131  port_init                         
00000200  __STACK_SIZE                      
000002bb  timer32_init                      
0000031b  main                              
00000459  SystemCoreClockUpdate             
000006d1  SystemInit                        
0000078d  CS_startLFXTWithTimeout           
00000829  __aeabi_memcpy                    
00000829  __aeabi_memcpy4                   
00000829  __aeabi_memcpy8                   
00000829  memcpy                            
000008c5  __aeabi_memclr                    
000008c5  __aeabi_memclr4                   
000008c5  __aeabi_memclr8                   
000008c7  __aeabi_memset                    
000008c7  __aeabi_memset4                   
000008c7  __aeabi_memset8                   
000008cd  memset                            
0000093f  __mpu_init                        
00000941  __TI_auto_init                    
000009b1  __TI_decompress_lzss              
00000a19  Interrupt_enableInterrupt         
00000a7d  _c_int00                          
00000ad1  C$$EXIT                           
00000ad5  abort                             
00000add  exit                              
00000b25  copy_in                           
00000b71  Interrupt_registerInterrupt       
00000ba5  _args_main                        
00000bbd  CS_setExternalClockSourceFrequency
00000bd1  _register_unlock                  
00000bd7  _register_lock                    
00000bdf  _nop                              
00000be5  SysCtl_A_disableNMISource         
00000bf5  SysCtl_A_enableNMISource          
00000c05  SysCtl_A_getNMISourceStatus       
00000c15  Timer32_registerInterrupt         
00000c25  __TI_decompress_none              
00000c33  Reset_Handler                     
00000c3f  ADC14_IRQHandler                  
00000c3f  AES256_IRQHandler                 
00000c3f  BusFault_Handler                  
00000c3f  COMP_E0_IRQHandler                
00000c3f  COMP_E1_IRQHandler                
00000c3f  CS_IRQHandler                     
00000c3f  DMA_ERR_IRQHandler                
00000c3f  DMA_INT0_IRQHandler               
00000c3f  DMA_INT1_IRQHandler               
00000c3f  DMA_INT2_IRQHandler               
00000c3f  DMA_INT3_IRQHandler               
00000c3f  DebugMon_Handler                  
00000c3f  Default_Handler                   
00000c3f  EUSCIA0_IRQHandler                
00000c3f  EUSCIA1_IRQHandler                
00000c3f  EUSCIA2_IRQHandler                
00000c3f  EUSCIA3_IRQHandler                
00000c3f  EUSCIB0_IRQHandler                
00000c3f  EUSCIB1_IRQHandler                
00000c3f  EUSCIB2_IRQHandler                
00000c3f  EUSCIB3_IRQHandler                
00000c3f  FLCTL_IRQHandler                  
00000c3f  FPU_IRQHandler                    
00000c3f  HardFault_Handler                 
00000c3f  MemManage_Handler                 
00000c3f  NMI_Handler                       
00000c3f  PCM_IRQHandler                    
00000c3f  PORT2_IRQHandler                  
00000c3f  PORT3_IRQHandler                  
00000c3f  PORT4_IRQHandler                  
00000c3f  PORT5_IRQHandler                  
00000c3f  PORT6_IRQHandler                  
00000c3f  PSS_IRQHandler                    
00000c3f  PendSV_Handler                    
00000c3f  RTC_C_IRQHandler                  
00000c3f  SVC_Handler                       
00000c3f  SysTick_Handler                   
00000c3f  T32_INT1_IRQHandler               
00000c3f  T32_INT2_IRQHandler               
00000c3f  T32_INTC_IRQHandler               
00000c3f  TA0_0_IRQHandler                  
00000c3f  TA0_N_IRQHandler                  
00000c3f  TA1_0_IRQHandler                  
00000c3f  TA1_N_IRQHandler                  
00000c3f  TA2_0_IRQHandler                  
00000c3f  TA2_N_IRQHandler                  
00000c3f  TA3_0_IRQHandler                  
00000c3f  TA3_N_IRQHandler                  
00000c3f  UsageFault_Handler                
00000c3f  WDT_A_IRQHandler                  
00000c41  __TI_zero_init                    
00000c4d  CS_startLFXT                      
00000c53  _system_pre_init                  
00000c57  _system_post_cinit                
00000c78  __TI_Handler_Table_Base           
00000c84  __TI_Handler_Table_Limit          
00000c98  __TI_CINIT_Base                   
00000cb0  __TI_CINIT_Limit                  
20000000  g_pfnRAMVectors                   
200000e8  __TI_cleanup_ptr                  
200000ec  __TI_dtors_ptr                    
200000f0  __TI_enable_exit_profile_output   
200000f4  _lock                             
200000f8  _unlock                           
200000fc  timer                             
20000100  status                            
20000104  main_func_sp                      
20000108  SystemCoreClock                   
2000fe00  __stack                           
20010000  __STACK_END                       
4000480c  WDTCTL_SYM                        
ffffffff  __TI_pprof_out_hndl               
ffffffff  __TI_prof_data_size               
ffffffff  __TI_prof_data_start              
ffffffff  __binit__                         
ffffffff  __c_args__                        
ffffffff  binit                             
UNDEFED   SHT$$INIT_ARRAY$$Base             
UNDEFED   SHT$$INIT_ARRAY$$Limit            

[123 symbols]
